:10200000120100020000004005164081000001029C
:1020100000010A06000200000040010009022E0033
:1020200001010080320904000004FF0000000705E0
:1020300002020002000705040200020007058602F2
:102040000002000705880200020009022E000101BB
:102050000080320904000004FF00000007050202AE
:10206000400000070504024000000705860240000A
:102070000007058802400000040309040C03410026
:10208000430043004500530026035500530042001F
:102090002D00410049004F00310036002D00310075
:1020A00036004100000000000000000000000000B9
:101A2E0060803E70013F01010101010700030202C7
:101A3E0002020200F5F7F7F7F7F7F7F700000000DC
:101A4E000000003F013F01010101010702050000F6
:101A5E0000000000F6F7F7F7F7F7F7F700000000C1
:101A6E000000003F011301210139010700010001AF
:101A7E00000B0200F7F7F3F7F5F7F7F7003600F073
:101A8E000012003F010138010101010702020D00A1
:101A9E0000000000F2F7F7F7F7F7F7F700002D0058
:101AAE000000003F60243EF7000000000000000030
:101ABE000000000000000000000000000000000018
:101ACE00000000000000000000000000473EF0E0B3
:101ADE008000F7AA4E0060803F1B013F010101010B
:101AEE0001070003020202020200F5F7F7F7F7F70B
:101AFE00F7F7000000000000003F013F0101010167
:101B0E0001070205000000000000F6F7F7F7F7F7EF
:101B1E00F7F7000000000000003F0113012101391A
:101B2E00010700010001000B0200F7F7F3F7F5F7CC
:101B3E00F7F7003600F0002D003F010138010101DA
:101B4E00010702020D0000000000F2F7F7F7F7F7A9
:101B5E00F7F700002D000000003F60243FA20000B8
:101B6E000000000000000000000000000000000067
:101B7E000000000000000000000000000000000057
:0C1B8E000000473F9BE08000F7AA4E00DB
:102A980090E67174FFF0F5B490E672E04480F0437C
:102AA800B6802290E60174AAF090E6F574FFF02251
:102AB800F59B759DE4E4F59EFF2290E67BE090E6A9
:042AC8007CF00F226D
:10215D00122AAB903F9BE090E6F3F0903F9CE0900D
:10216D00E6C3F0903F9DE090E6C1F0903F9EE09079
:10217D00E6C2F0903FA0E090E6C0F0903FA1E09065
:10218D00E6F4F075AF07743FF59A741B122AB81276
:10219D002AC2BF80FA122A98000000E490E6C4F02B
:1021AD0000000090E6C5F0903FA2E090E6C6F090EA
:1021BD003FA3E090E6C7F0903FA4E090E6C8F09012
:1021CD003FA5E090E6C9F0903FA6E090E6CAF090FA
:1021DD003FA7E090E6CBF0903FA8E090E6CCF090E2
:0821ED003FA9E090E6CDF022CD
:1021F500122AAB903EF0E090E6F3F0903EF1E090CD
:10220500E6C3F0903EF2E090E6C1F0903EF3E09038
:10221500E6C2F0903EF5E090E6C0F0903EF6E09024
:10222500E6F4F075AF07743EF59A7470122AB81289
:102235002AC2BF80FA122A98000000E490E6C4F092
:1022450000000090E6C5F0903EF7E090E6C6F090FD
:102255003EF8E090E6C7F0903EF9E090E6C8F090D1
:102265003EFAE090E6C9F0903EFBE090E6CAF090B9
:102275003EFCE090E6CBF0903EFDE090E6CCF090A1
:082285003EFEE090E6CDF022E0
:0A2F31000001020203030404050579
:102B3200EC4EFEED4F2431F582742F3EF583E49383
:102B4200FF3395E0FEEF24A1FFEE34E68F82F5839A
:102B52002290E6BCE0547EFF7E00E0D394807C00AD
:012B62002250
:10228D00E4F530F52FF52EF52DC20CC209C20BC2A7
:10229D000A12140F750A20750B0075122075131292
:1022AD0075082075091C75102075114A7514207557
:1022BD001578D2E843D82090E668E04409F090E61E
:1022CD005CE0443DF0D2AFD20F122B6390E680E07C
:1022DD0054F7F0538EF8C20C300A05121884C20A56
:1022ED00300C29122EB55024C20C122C8120091647
:1022FD0090E682E030E704E020E1EF90E682E03006
:10230D00E604E020E0E4122B92122EC7121CD780B7
:01231D00C7F8
:1018840090E6B9E070030219351470030219892433
:10189400FE70030219E324FB700302192F14700372
:1018A40002192914607314607624056003021A1A5D
:1018B400121EFE4003021A2690E6BBE024FE6022BC
:1018C40014603324FD601114602224067048E50A74
:1018D40090E6B3F0E50B8037E51290E6B3F0E5133C
:1018E400802DE50C90E6B3F0E50D8023E50E90E63F
:1018F400B3F0E50F801990E6BAE0FF122BBEAA06FA
:10190400A9077B01EA494B600DEE90E6B3F0EF9036
:10191400E6B4F0021A26021A1F122F4F021A2612D8
:101924002F45021A26122971021A26122F3B021A77
:1019340026121FFE4003021A2690E6B8E0247F60B8
:10194400151460192402703AA209E43325E0FFA2B9
:101954000BE4334F8018E490E740F08016122B53C9
:1019640040047D0180027D00122B32E0540190E797
:1019740040F0E4A3F090E68AF090E68B7402F00263
:101984001A26021A1F122FB44003021A2690E6B830
:10199400E024FE601624026003021A2690E6BAE0F0
:1019A400B40105C209021A26021A1F90E6BAE070B1
:1019B4002C122B5340047D0180027D00122B32E057
:1019C40054FEF090E6BCE05480131313541FFFE060
:1019D400540F2F90E683F0E04420F08045803C12C1
:1019E4002FB6503E90E6B8E024FE601A240270320E
:1019F40090E6BAE0B40104D209802790E6BAE0B4D4
:101A04000202801E8015122B5340047D0180027D4A
:101A140000122B328008120080500790E6A0E044A8
:0A1A240001F090E6A0E04480F022FB
:03003300022F9EFB
:042F9E0053D8EF32E3
:100C47000D2020455030200020526561643A200075
:100C570057726974653A200030780020563A307828
:100C6700002C20493A3078002C204C3A3078000D7F
:100C77002020455030425546203D20307800202125
:100C87003D20004020504F535420002D2050415309
:100C970053200D002D204641494C200D000A0A0A19
:100CA7000A0A0D5553422D41494F20262044504BE7
:100CB7002D41494F2046616D696C79204669726DF7
:100CC700776172650D007573622D61696F31362D1D
:100CD7003136412E63204D6172203330203230315E
:100CE7003520402031383A35393A32330D0040202B
:100CF70054445F494E49542053544152540D0036D1
:100D07002D31364100362D31364500322D313641F1
:100D170000322D313600322D31364500362D36342E
:100D27004D4100362D36344D4500322D36344D4178
:100D370000322D36344D00322D36344D4500362DD8
:100D470033324100362D33324500322D33324100E4
:100D5700322D333200322D33324500362D363441B1
:100D670000362D36344500322D36344100322D36CB
:100D77003400322D36344500362D39364100362DB4
:100D870039364500322D39364100322D3936003299
:100D97002D39364500362D3132384100362D313266
:100DA700384500322D3132384100322D313238008A
:100DB700322D31323845002D4F54484552006D735E
:100DC7000D00210054445F504F4C4C3A2047504986
:100DD7004654524947202620307838300D005F00AE
:100DE700475049464D6F64655365743A0020434F39
:100DF7004E54494E554F55530D002054430D000D89
:100E07003D20002D2072652D72756E6E696E67200C
:100E170054445F494E4954002D2054445F494E497C
:100E2700542072652D72756E20646F6E652E002DCD
:100E3700203078424320577269746520002D205076
:100E470069636B47504946203D2000436F6E7469C4
:100E57006E756F757320005443204D6F64652000D5
:100E67002D2057726974652034303146203D20307B
:100E770078002D2054436F756E74203D2030780024
:100E87002D204144435F436F6E74696E756F7573B0
:100E97003D002D203078424320526561643A20009E
:100EA7002D20435452526561640D002D2043545246
:100EB7004D6F646520004354522000203D204D4F64
:100EC700444520002D204354524C6F6164200D008F
:100ED7002D204354524D6F64654C6F616420002090
:100EE7004C6F6164203D203078002D2044494F57D6
:100EF70072697465416C6C3A002D2044494F5F520A
:100F0700656164416C6C3A002D2044494F5F436F23
:100F17006E6669677572653A002D204144435F53D9
:100F27006574436F6E6669673A002D204144435FDD
:100F3700476574436F6E666967002D2030784246B7
:100F47003A476574496D6D6564696174652000533E
:100F57007461727420312041444320436F6E76657B
:100F67007273696F6E200054616B652032204144B3
:100F7700432C206672657368206461746120005495
:100F8700616B652031204144432C20686973746F7D
:100F9700726963616C206461746120002D20536560
:100FA7006C6620546573743A002D205041535300EA
:100FB7002D204641494C000D002D2050726F62656F
:100FC7002043616C3A002D20537570706F72746501
:100FD7006420002D20556E617661696C61626C65D5
:100FE700002D2057726974652043616C200D002E17
:100FF7000020756E617661696C61626C652E002DEB
:101007002056525F4E4F5344504155544F002D20A8
:10101700444F204E4F542057414E54002D205652D6
:101027005F52414D20262056525F454550524F4D45
:101037000D002D20444143536574426F6172645221
:10104700616E6765002D203078423420414F20447F
:101057004143002D20307842332044414344697294
:10106700656374200D002D203078423320444143BE
:101077004D756C74694469726563743A20002D205C
:1010870030784233205348454E414E4947414E53ED
:10109700204C656E6774683D3078002D2054445F9E
:1010A70053757370656E640D002D2054445F52654F
:1010B70073756D650D002D205265736574003600DC
:1010C70049424E00706E360065663200656636002E
:1010D7004646320046463600436F6E74005443203E
:0210E7002000E7
:101B9A00413FCA00413FD0FF413FCBFE413FE900F0
:101BAA00413FD300024E0000C104C106C102C10870
:101BBA00C103C101413FCCFB413FCD50024C000063
:021BCA00C10058
:1016B5007A0D792A7BFFE4F545754601227A0D7985
:1016C500237BFF75450175460122E490E68AF0907B
:1016D500E6BEE090E68BF02290E6BAE075F008A44D
:1016E500FFA3E07C002FFFEC35F0FEE42FF58274BC
:1016F500503EF583E02290E678E04401F0E0541096
:10170500FFC4540F4450903FC9F0E013E433903FB9
:10171500D2F022E090E740F0E490E68AF090E68B84
:10172500227A0D790C7BFFE4F545F54622FF90E61C
:10173500BAE075F008A42403F582E5F03450F5838A
:10174500EFF022AD3A7AE779407F40AB072274D4B7
:101755002FF582E4343FF583E4F02FF582E434403D
:10176500F5832290E6BCE0FF90E6BBE022744025BD
:101775003CF582E434E7F583222536F536E539353F
:1017850035F535C3E538953AF538E5379539F53703
:10179500227A0D79067BFF754501E4F546227586AB
:1017A500005391EF90E65D22903FD0EFF0E0FF44CB
:1017B5004090200AF0EF541F2290E740E09040153A
:1017C500F090E741E0904016F022904017E090E756
:1017D50040F0904018E090E741F0227A0D791D7BAA
:1017E500FFE4F545F54622C3E53C953AE53B9539D9
:1017F5002290E6047480F0223EF583E0FBED25E0BF
:10180500FFEC33FE22E536253CF582E535353BF523
:10181500832290E6BEE0D394002290E6C37480F064
:1018250090E6C214F022F582E4343FF5832290E677
:1018350084E0FE90E685E0FD2274412FF58274E791
:101845003EF58322850D82850C83A37402F02285E3
:101855000F82850E83A37407F022F07A3F7BEAADF1
:10186500407F0E22FEE07C002400FFEC3E22E49047
:0F187500E68AF090E6BEE0225391EF90E65B2208
:102C1100754003903FEA7430F0E4A3F0A37403120B
:102C2100185F122E0E903FEA7438F0E4A3F0A3046B
:062C310012185F022E0ED6
:0C2F2500C007EDAD03FCEBD00702261145
:1023AA007BFF7A0C79471229B390E6B8E07BFF30BD
:1023BA00E7067A0C794F80047A0C79571229B37B95
:1023CA00FF7A0C795F1229B390E6B9E0FF122ED991
:1023DA007BFF7A0C79621229B390E6BBE0FF122EDA
:1023EA00D990E6BAE0FF122ED97BFF7A0C796812EF
:1023FA0029B390E6BDE0FF122ED990E6BCE0FF12A9
:10240A002ED97BFF7A0C796F1229B390E6BFE0FFD1
:10241A00122ED990E6BEE0FF122ED97F0D022E7E33
:10286500E4FBFA12181740367BFF7A0C79761229A9
:10287500B3E4FAFB90E6BEE0FFC3EB9F7480F86A11
:1028850098501B74402BF58274E73AF583E0FF12EC
:102895002ED97F20122E7E0BBB00010A80D6300F69
:0528A50003122F99222F
:042FA2004380022244
:042FA6005380FD2235
:042FAA00638002221C
:102E91001217F60000007406F0000000E4F00000D4
:022EA10000220D
:102E2A00C20890E61474E0F000000090E61A7409F3
:072E3A00F0000000022E91E0
:102EA3001217F60000007402F0000000E4F00000C6
:022EB3000022FB
:1028ED0090E61274A0F000000090E6187411F0004C
:1028FD000000122EA390E6917480F0000000F0000D
:10290D000000F0000000F000000090E6497482F035
:10291D00000000F0000000F0000000F000000002D8
:02292D002EA3D7
:062F8E001228ED022E2ABC
:102D1200D205904011E4F090401C04F0E4F075B349
:102D2200FF90E671F075B4FF75B5FF90E672F0752D
:032D3200B6FF22C7
:082F7E00D205E4F5B3F5B5221C
:102D3500C205903FE5E0904011F0E4F5B390E671EF
:102D450074FFF0F5B4E4F5B590E6727480F075B6ED
:022D5500FF225B
:102CA600E4FEFD7801AF05EF08800103D8FDF5B11C
:102CB6008DB08EA08E9090401BEEF00EEE70E40D5F
:042CC600ED70E022AB
:10249400E4F543FC7801AF04EF08800103D8FDF5AF
:1024A400B18543A090401C7401F085904185B042F1
:1024B400E4F0E541B54305E5426C6028903FCB74F8
:1024C40001F0AF04122ED9AF43122ED97BFF7A0C40
:1024D40079851229B3AF42122ED9AF41122ED912E7
:1024E4002F9980060543E54370AA0CEC70A6903F33
:0824F400CBE0B4FE02E4F0228B
:10292F007BFF7A0C798A1229B3122D129040107402
:10293F0001F0122CA69040107405F0122CA6122F45
:10294F007E122494122D35903FCBE07BFF70067AD8
:10295F000C799280047A0C799B1229B3904010E481
:02296F00F02254
:1025BA008B478A488949E4F54A122E418F4BE54BED
:1025CA0025E02410902088F0E4F54AAF4BEF3395CC
:1025DA00E0FEC3E54A9FEE6480F87480985027AB0A
:1025EA0047AA48A949854A82758300121DEBFDE571
:1025FA004A75F002A42498F9742035F08982F5838B
:07260A00EDF0054A80C52236
:102BEA0090401374AAF0E064AA70197455F0E06476
:102BFA00557011744FF0E0B44F0A7449F0E0B449CB
:072C0A00037F00227F01227D
:10242A00122BEAEF14601B04705A12174A7D017FBF
:10243A00037E0012266590E740E0541F903FD0F0DB
:10244A00804212174A7D027FF67E1D12266590E7AA
:10245A0040E0FF780208800123D8FDF54190E7416A
:10246A00E0903FD0F012174A7D017F037E001226CA
:10247A006590E740E0654160037F042290E740E011
:0A248A00541FFF22903FD0E0FF2214
:102E560090401AEDF0903FE9E545F0903FD3E54606
:042E6600F00225BA97
:10140F00E4F540122EFA7BFF7A0C79A41229B37BF4
:10141F00FF7A0C79CD1229B37BFF7A0C79F512295B
:10142F00B390E6017480F0122F861216FB90E6003F
:10143F007410F090E61074A0F090E611F000000028
:10144F0090E612F0000000E490E613F00000009028
:10145F00E61474E0F0000000E490E615F01217F6C1
:10146F000000007482F00000007486F0000000E4B9
:10147F00F000000090E618F00000007411F000007A
:10148F000090E61A7409F000000012242A1217AD1A
:10149F00B41E00400302167F9014AEF82828730282
:1014AF00150802150F02151702152302152F021525
:1014BF003702153F02154702155302155F02156DCE
:1014CF0002157B0215890215970215A50215B302A5
:1014DF0015C10215CF0215DD0215EB0215F9021623
:1014EF000702161402162102162E02163B02164888
:1014FF0002165502166202166F121796FD02167A21
:10150F001217267D0102167A7A0D791212179A7D1B
:10151F000202167A7A0D791812172A7D0302167AAB
:10152F001217E07D0402167A1216C27D0802167A8F
:10153F001216B57D0902167A7A0D79311216C67D0B
:10154F000A02167A7A0D79381216B97D0B02167ABD
:10155F007BFF7A0D793E1216BB7D0C02167A7BFF4C
:10156F007A0D79451216C87D1002167A7BFF7A0D17
:10157F00794B1216BB7D1102167A7BFF7A0D7951CA
:10158F001216C87D1202167A7BFF7A0D7957121642
:10159F00BB7D1302167A7BFF7A0D795C1216BB7D29
:1015AF001402167A7BFF7A0D79621216C87D10022B
:1015BF00167A7BFF7A0D79681216BB7D1102167AA7
:1015CF007BFF7A0D796E1216C87D1202167A7BFF99
:1015DF007A0D79741216BB7D1302167A7BFF7A0D82
:1015EF0079791216BB7D1402167A7BFF7A0D797FFB
:1015FF001216C87D1002167A7BFF7A0D79851216A6
:10160F00BB7D1180667BFF7A0D798B1216C87D1218
:10161F0080597BFF7A0D79911216BB7D13804C7B1D
:10162F00FF7A0D79961216BB7D14803F7BFF7A0DE2
:10163F00799C1216C87D1080327BFF7A0D79A31228
:10164F0016BB7D1180257BFF7A0D79AA1216C87DF6
:10165F001280187BFF7A0D79B11216BB7D13800BA8
:10166F007BFF7A0D79B71216BB7D14122E568009A7
:10167F007BFF7A0D79BE1225BAE4FF121753E4F0FF
:10168F000FBF15F790401DE4F012292FC210122D35
:10169F00D512181F00000090E6E27402F043B20268
:0616AF00D2097550012272
:1010E900E4F51C122EFA7BFF7A0C79A41229B37B42
:1010F900FF7A0C79CD1229B37BFF7A0C79F5122985
:10110900B3121833EEF51DEDF51ED204C206C2075F
:10111900C205C208C203C20190401FE4F012181FA1
:1011290090E600E054E74410F090E6017480F090F6
:10113900E67AE04401F0122F861216FB90E610744D
:10114900A0F000000090E611F0000000E490E61322
:10115900F000000090E615F0000000122F8E122416
:101169002A1217ADB41E00400302135390117CF8E4
:101179002828730211D60211DD0211E50211F302CA
:1011890011FF02120702120F021217021225021290
:101199003302124102124F02125D02126B021279DE
:1011A9000212870212950212A30212B10212BF02A1
:1011B90012CD0212DB0212E80212F5021302021327
:1011C9000F02131C02132902133602134312179636
:1011D900FD02134E1217267D0102134E7BFF7A0D75
:1011E900791212179C7D0202134E7A0D7918121783
:1011F900E47D0302134E1217E07D0402134E12160A
:10120900C27D0802134E1216B57D0902134E7BFFEB
:101219007A0D79311216C87D0A02134E7BFF7A0DB9
:1012290079381216BB7D0B02134E7BFF7A0D793E7E
:101239001216BB7D0C02134E7BFF7A0D79451216EF
:10124900C87D1002134E7BFF7A0D794B1216BB7DB8
:101259001102134E7BFF7A0D79511216C87D1202C5
:10126900134E7BFF7A0D79571216BB7D1302134E6D
:101279007BFF7A0D795C1216BB7D1402134E7BFF3E
:101289007A0D79621216C87D1002134E7BFF7A0D12
:1012990079681216BB7D1102134E7BFF7A0D796EA8
:1012A9001216C87D1202134E7BFF7A0D797412163D
:1012B900BB7D1302134E7BFF7A0D79791216BB7D24
:1012C9001402134E7BFF7A0D797F1216C87D100226
:1012D900134E7BFF7A0D79851216BB7D1180667BD3
:1012E900FF7A0D798B1216C87D1280597BFF7A0D12
:1012F90079911216BB7D13804C7BFF7A0D7996127A
:1013090016BB7D14803F7BFF7A0D799C1216C87D30
:101319001080327BFF7A0D79A31216BB7D118025CF
:101329007BFF7A0D79AA1216C87D1280187BFF7A85
:101339000D79B11216BB7D13800B7BFF7A0D79B73E
:101349001216BB7D14122E5680097BFF7A0D79BEC9
:101359001225BAE4FF121753E4F00FBF15F79040B6
:101369001DE4F012292FC210122DD590E6E2740265
:10137900F000000043B202D20990E65EE04450F06A
:1013890000000090E65AE04450F000000090E65852
:10139900E04450F000000090E650E04403F0000003
:1013A9000090E654E04403F0000000121833EDF514
:1013B900828E837F20122E7EAF82122F0A7F2D12FA
:1013C9002E7EAF1EAE1D122F0A7F3D122E7EC3E563
:1013D90082951EFFE583951DFED3E51E9582E51DC9
:1013E900958350067C007D0080047C087D00EF2DEC
:1013F900FFEE3CFE122F0A7BFF7A0D79C51229B345
:06140900755001D204221F
:101CD700E58070047F0180027F00EF90E68030E0AE
:101CE70006E04408F08004E054F7F0E55070033054
:101CF7000035E54D454C7006754C08754DFFE54DB3
:101D0700154D7002154CE54D454C7004F550800F8C
:101D1700AE4CAF4D7C027D3F121E3AEF20E005121C
:101D27002FA68003122FA230084C90401FE030E00E
:101D370045C2087BFF7A0D79C91229B390401FE489
:101D4700F090E6F574FFF0C2061217F6E490E6CEBF
:101D5700F000000090E6CFF000000090E6D0F00021
:101D6700000090E6D1F000000090E604F0000000CB
:101D7700122E91122FAA300851E5BB30E74C7BFF9A
:101D87007A0D79CB1229B300000090E6AFE090E618
:101D9700B0121869FED3EF9400EE9400400EEE9453
:101DA70002500990E6487406F0000000122F0A7BE3
:101DB700FF7A0D79E51229B390E698E0FF122ED944
:0B1DC70090E699E0FF122ED9C208221E
:1020B000E4FF9040117404F0A374F0F0A37401F0F5
:1020C000E490E6CEF000000090E6CFF00000009033
:1020D000E6D0F000000090E6D17420F0000000751A
:1020E000BB06000000904019E4F01FEF600AE5BB5A
:1020F00020E70500000080F2E4FDFCEDAE0478026C
:10210000C333CE33CED8F92402F58274F81217FD0A
:1021100074402FF58274E73EF583EBF0EDAE047862
:1021200002C333CE33CED8F92403F58274F81217E4
:10213000FD12183EEBF00DBD00010CED64104C706B
:10214000BA122E91903FE5E0904011F0903FE6E00A
:0D215000904012F0903FE7E0904013F02225
:1024FC00E4FF9040117404F0904013E4F090401EFF
:10250C007481F0E490E6CEF000000090E6CFF0008D
:10251C00000090E6D0F000000090E6BEE0C31390FF
:10252C00E6D1F075BB06000000904019E4F01FEFF7
:10253C00600AE5BB20E70500000080F2E4FF90E6AE
:10254C00BEE0FEEFC39E500B74402F121776E4F0E2
:06255C000F80EB022E913E
:10008000E4F53DF53E75500120030B90E6B9E064C0
:10009000D460031223AA30030A90E6B9E0B4BE0389
:1000A0001223AA90E6B9E0121E8F04AE1004C2110A
:1000B00004E21203762003CF2103E02203F023069B
:1000C000EC3506E638011639077891096FA2096FF9
:1000D000A30962A9092FAC0AEAB30ACBB40102B69C
:1000E0000AA1B707ABBA07E7BB01BABC0500BE0659
:1000F000F2BF0104C30500D2014FD40ACBFB0000BC
:100100000B9D800C121768FD90E6BAE0FB122F25BC
:100110001220B002079C90E6B8E020E7307A0D7913
:10012000E7120C077BFF60067A0D79F480047A0EE3
:1001300079011229B390E6BCE0600A146003020B57
:100140009FD20F8002C20F122F59020B9F8059902D
:10015000E6B8E020E75290E6BFE0FF90E6BEE04F51
:10016000600A1216CF90E6A0E020E1F97A0E790637
:10017000120C07B48102D20890E6BCE0B48002C23F
:100180000890E6BCE0B413147BFF7A0E790A1229BA
:10019000B312140F7BFF7A0E791F80067B017AE77A
:1001A00079401229B3020B9F90E6BCE0FFE42F12C6
:1001B0001760E090E740F0020AAB90E6B8E030E765
:1001C000030202E47BFF7A0E79361229B3D20112C0
:1001D0001817400F1216CF90E6A0E020E1F9C20FE9
:1001E00012286590E6BEE0C39404404D90E740E0DD
:1001F00030E2297BFF7A0E79441229B390E743E07D
:100200007BFF30E0067A0E795280047A0E795E1216
:1002100029B390E743E013920F122F5990E740E083
:1002200030E1167BFF7A0E79671229B390E742E03E
:10023000FF122ED9E090401FF090E6BEE0600A90D9
:10024000E740E020E0030202DC7BFF7A0E797912BE
:1002500029B390E6BBE0FF122ED990E6BAE0FF1278
:100260002ED9120BE6E5AC5401FFE5BB54804F904C
:10027000E740F0E030E765E020E0611217684FFFEB
:1002800090E6BDE04FFF90E6BAE04F7003D38001E7
:10029000C392067BFF7A0E79871229B3A206E43354
:1002A000FF122ED990E6BBE090E6CEF00000009061
:1002B000E6BAE090E6CFF000000090E6BDE090E600
:1002C000D0F0000000A206E433FF90E6BCE04F90BF
:1002D000E6D1F000000075BB06000000122F99D295
:1002E00008020B9F7BFF7A0E79991229B390E6B032
:1002F000E090E740F090E6AFE090E741F090E699BB
:10030000E090E742F000000090E698E090E743F0CC
:1003100000000090E614E090E744F090E61AE090C8
:10032000E745F000000090E635E090E746F0000079
:100330000090E634E090E747F0000000A3E5ACF061
:1003400090E6A9E090E749F090E654E090E74AF0A3
:1003500000000090E655E090E74BF0000000300709
:10036000047F0180027F0090E760EFF0E490E68A6E
:10037000120C2C0209227A0E79A7120C33B4020E49
:1003800090E6BBE0C4333354C0121732802690E6A7
:10039000BEE06403701E90E6BBE0FF7401A807088E
:1003A0008002C333D8FC25E044C01217321216DD98
:1003B00090E742F01216DD90E740F090E6BAE07563
:1003C000F008A4FFA3E01216EA90E7410206E07AE3
:1003D0000E79B2120BB4120C11120BF7F0020B9F34
:1003E0007BFF7A0E79CB1229B3E490E68B020426C8
:1003F00090E6B8E030E703020B9F90E6BFE07004A0
:100400007F0180027F0090E6BEE04F60467A0E7961
:10041000D7120BB4120C117BFF7A0E79E61229B3B6
:10042000120BE6120BF7F0121768C4131354037C77
:10043000005403FDE42DF582EC12174190E6BD1245
:10044000176BC413135403FDE42DF582EC1217410E
:10045000020B9F90E6BEE06408701C1216D090E676
:10046000A0E020E1F9744044E76003020B9F905044
:10047000037474F0020B9F90E6BEE0640460030214
:100480000B9F9050037474F074B4F090E742E090C6
:100490005002F090E743E0905002F090E740E09087
:1004A0005001F090E741E0905001F0020B9F7A0E6E
:1004B00079F1120BA190E6A0E020E1F91217BE023B
:1004C00006287BFF7A0F79001229B3904015E0903F
:1004D000E740F0904016E090E741F0E490E68A02B1
:1004E00006E07A0F790F120BA190E6A0E020E1F967
:1004F00090E742E05403904014F01217BE020B9FA5
:1005000090E6B8E030E7030206307BFF7A0F7920EF
:100510001229B3C2031216CF90E6A0E020E1F990B1
:10052000E740E0903FD4F0904000F090E741E09049
:100530003FD5F0904001F090E742E0903FD6F09038
:100540004002F090E743E0903FD7F0904003F090F6
:10055000E744E0903FD8F0904004F090E745E09009
:100560003FD9F0904005F090E746E0903FDAF090F8
:100570004006F090E747E0903FDBF0904007F090B6
:10058000E748E0903FDCF0904008F090E749E090C9
:100590003FDDF0904009F090E74AE0903FDEF090B8
:1005A000400AF090E74BE0903FDFF090400BF09076
:1005B000E74CE0903FE0F090400CF090E74DE09089
:1005C0003FE1F090400DF090E74EE0903FE2F09078
:1005D000400EF090E74FE0903FE3F090400FF09036
:1005E000E750E0903FE4F0904010F090E751E09049
:1005F0003FE5F0904011F090E752E0903FE6F09038
:100600004012F090E753E0FF903FE7F0904013F086
:10061000903FD0E0541FD39404400D90E754E0FF86
:10062000903FE8F090401DF0D20F122865020B9F1A
:100630007BFF7A0F79311229B3903FD4E090E740E5
:10064000F0903FD5E090E741F0903FD6E090E74250
:10065000F0903FD7E090E743F0903FD8E090E74438
:10066000F0903FD9E090E745F0903FDAE090E74620
:10067000F0903FDBE090E747F0903FDCE090E74808
:10068000F0903FDDE090E749F0903FDEE090E74AF0
:10069000F0903FDFE090E74BF0903FE0E090E74CD8
:1006A000F0903FE1E090E74DF0903FE2E090E74EC0
:1006B000F0903FE3E090E74FF0903FE4E090E750A8
:1006C000F0903FE5E090E751F0903FE6E090E75290
:1006D000F0903FE7E090E753F0903FE8E090E75478
:1006E000120C2C0207A490E6F574FFF0122E910272
:1006F0000B9F7A0F7941120C3370247BFF7A0F79AC
:10070000561229B3904018E0FF122ED9904017E0FE
:10071000FF122ED9122F99904019E4F0020B9790F6
:10072000E6BEE064047BFF70327A0F796E1229B363
:10073000904019E4F01217CF904019E4F090401760
:10074000E090E742F0904018E090E743F0D20F12BB
:10075000286590E68B7404F0020B9F7A0F7986125D
:1007600029B31217CFD20F12286590E68B7402F0CE
:10077000904019E4F0020B9F7BFF7A0F79A31229B6
:10078000B3903FCBE0FF90E740F0EF7BFF70067A3D
:100790000F79B080047A0F79B7120C1F90E6BFE092
:1007A00090E68AF090E6BEE0020B977BFF7A0F7925
:1007B000C01229B3903FE9E0FFB4010890E740740C
:1007C000BBF08008903FD0E090E740F0EF7BFFB4B3
:1007D00001067A0F79CD80047A0F79DA120C1F1294
:1007E000171D04F0020B9F90E6B8E030E71990E681
:1007F000BEE0B4011290E7407401F012292F90E698
:100800008B7401F0020B9F7BFF2003127A0F79E8B3
:100810001229B3D203C20F122F59C20180077A0FD7
:1008200079F61229B3903FE9E064016003020909F7
:10083000122D3590E74074BBF090E6BBE0C313FF88
:10084000E5B154802FF5B1E090E6C4F090E6BAE04F
:1008500090E6C5F090E6BDE090E6BC121869903FC6
:10086000CEF0A3EFF0903FCEE0FEA3E0FF4E70038A
:10087000020904E5BB30E7EDE5AB20E1E830044CCC
:10088000D3EF9400EE9402401C90E6D07402F00086
:100890000000E490E6D1F0000000903FC67402F042
:1008A000A3E4F08027903FCEE0FCA3E0FDEC90E6CF
:1008B000D0F0000000ED90E6D1F0000000903FCEB7
:1008C000E0FFA3E0903FC6CFF0A3EFF0E4F5BB005C
:1008D0000000E5BB20E7030080F800000000009066
:1008E0003FC6E0FEA3E0FFC3903FCFE09FF0903F04
:1008F000CEE09EF0E5B1547F04FFE5B154802FF5C2
:10090000B1020865122F7E80117BFF7A0F79F812F1
:1009100029B3903FD0E090E740F090E6BFE090E64A
:100920008AF01216D490E6A0E04480F0020B9F7B80
:10093000FF7A1079061229B37BFF7A1079151229F4
:10094000B390E6B5E054FEF090E6BFE01216D0900A
:10095000E6BBE090E6B3F090E6BAE090E6B4F002D1
:100960000B9F903FD27401F0903FC9E04401F07BAF
:10097000FF7A1079231229B390E6BAE0753500F5B5
:1009800036A3E0FEEE423590E6BEE0753700F5385E
:10099000A3E0FEEE423790E6B8E064C06003020ACE
:1009A00042E53845377003020B9F90E6A0E020E156
:1009B000F9C3E5389440E537940050088537398508
:1009C000383A8006753900753A4090E6B9E064A37C
:1009D000704090E6BCE0B4011BA3E0701790E6BB4A
:1009E000E030E71090E7407403F0A37401F0A374C3
:1009F00007F08042E4F53BF53C1217EC5038121832
:100A00000AE0FF121772EFF0053CE53C70EB053B86
:100A100080E7E4F53BF53C1217EC501012177274A6
:100A2000CDF0053CE53C70EF053B80EB121748AF7D
:100A300036AE3512266512171DE53AF012177E0202
:100A400009A190E6B8E064406003020B9FE53845D9
:100A5000377003020B9F12171DF090E6A0E020E113
:100A6000F990E68BE0753900F53A90E6B9E0B4A369
:100A70001EE4F53BF53C1217EC501E121772E0FF16
:100A800012180AEFF0053CE53C70EB053B80E712DD
:100A90001748AF36AE35122A63E53A12177E020ABE
:100AA0004D7A107939120C3D30E706121873020B9B
:100AB000971218174005E090E68BF0903FCAE0448B
:100AC0008090401EF0122C11020B9F7A10794C126C
:100AD0000C3D20E70F1216CF90E6A0E020E10302C4
:100AE0000B9F80F4121873020B9790E6BEE0701B08
:100AF0007BFF7A10795A1229B31216D4121768FDA7
:100B000090E6BAE0FB122F25020B9F90E6BEE06450
:100B100011706A7BFF7A10796D1229B31216CF908B
:100B2000E6A0E020E1F9D20F122865E4F53BF53CA0
:100B300090E740E0F53FE53F6065C3E53C9402E5A2
:100B40003B9400505AE53F30E023AF3CC007E53C02
:100B500025E0FFE53B33FE74422FF58274E73EF556
:100B600083E0FD12183EE0FBD007122F25053CE57F
:100B70003C7002053BE53FC313F53F80B97BFF7A2C
:100B80001079851229B390E6BFE0FF122ED990E6C6
:100B9000BEE0FF122ED9E090E68BF08002D322C394
:100BA000227BFF1229B3E490E68AF090E6BEE09043
:100BB000E68BF0227BFF1229B390E6BBE0FFC41363
:100BC000135403753D005403F53E7BFF7A0E79BD47
:100BD0001229B3AF3E122E6A7BFF7A0E79C2122918
:100BE000B390E6BBE02290E6BDE0FF122ED990E67E
:100BF000BCE0FF122ED922122F99E490E68BF090E0
:100C0000E6BBE0905003227BFF1229B390E6BCE0E4
:100C100022C313753D005407F53EFF122E6A2212BF
:100C200029B37BFF7A0F79BE1229B322F0D20F12BB
:100C30002865227BFF1229B390E6BEE0227BFF12DB
:070C400029B390E6B8E022A1
:102EB5007BFF7A1079A21229B37F017E0012281FA9
:022EC500D32216
:102EC7007F017E0012281F7BFF7A1079B01229B389
:022ED700D32204
:021EFE00D322ED
:1029710090E680E030E71800000090E6247402F051
:10298100000000E490E625F0000000D2048016006B
:102991000000E490E624F000000090E6257440F089
:1029A100000000C20490E6BAE0903FD1F0122F99E6
:0229B100D3222F
:0A2F3B00903FD112171804F0D322C2
:0A2F450090E6BAE0903FC8F0D322F6
:0A2F4F00903FC812171804F0D322B7
:021FFE00D322EC
:022FB400D32226
:022FB600D32224
:102CCA00C0E0C083C082C085C084C086758600D239
:102CDA000A1217A67401F0D086D084D085D082D08B
:042CEA0083D0E03281
:102D7900C0E0C083C082C085C084C0861217A37416
:0F2D890004F0D086D084D085D082D083D0E032C1
:102D9800C0E0C083C082C085C084C0861217A374F7
:0F2DA80002F0D086D084D085D082D083D0E032A4
:10256200C0E0C083C082C085C084C086758600C0BA
:10257200D075D000C000C001C002C003C0078510E2
:102582000C85110D12184985080E85090F12185471
:102592001217A67410F07BFF7A1079BD1229B3D0FE
:1025A20007D003D002D001D000D0D0D086D084D0C2
:0825B20085D082D083D0E03215
:102CEE00C0E0C083C082C085C084C086758600D215
:102CFE000C1217A67408F0D086D084D085D082D05E
:042D0E0083D0E0325C
:1029F200C0E0C083C082C085C084C0867586009056
:102A0200E680E030E71285080C85090D1218498529
:102A1200100E85110F1218541217A67420F0D086CA
:0B2A2200D084D085D082D083D0E03279
:012FB80032E6
:012FB90032E5
:012FBA0032E4
:012FBB0032E3
:012FBC0032E2
:012FBD0032E1
:102C3700C0E0C083C082C085C084C086758600534B
:102C470091EF90E65F7410F0D086D084D085D08263
:052C5700D083D0E03243
:012FBE0032E0
:101EB500C0E0C083C082C085C084C086758600C06E
:101EC500D075D000C000C001C002C003C007539147
:101ED500EF90E65F7440F07BFF7A1079C51229B365
:101EE500D007D003D002D001D000D0D0D086D08486
:091EF500D085D082D083D0E03208
:012FBF0032DF
:101FB800C0E0C083C082C085C084C086758600C06A
:101FC800D075D000C000C001C002C003C0071218FD
:101FD8007D7401F07BFF7A1079C71229B3D007D03E
:101FE80003D002D001D000D0D0D086D084D085D004
:061FF80082D083D0E0322C
:012FC00032DE
:012FC10032DD
:102D5700C0E0C083C082C085C084C086758600126B
:102D6700187D7410F0D086D084D085D082D083D0DF
:022D7700E03248
:012FC20032DC
:1027D900C0E0C083C082C085C084C086758600C041
:1027E900D075D000C000C001C002C003C0071218D4
:1027F9007D7440F07BFF7A1079CB1229B3D007D0D2
:1028090003D002D001D000D0D0D086D084D085D0DA
:0628190082D083D0E03202
:012FC30032DB
:012FC40032DA
:012FC50032D9
:012FC60032D8
:012FC70032D7
:012FC80032D6
:012FC90032D5
:012FCA0032D4
:012FCB0032D3
:012FCC0032D2
:1026B500C0E0C083C082C085C084C086758600C066
:1026C500D075D000C000C001C002C003C00753913F
:1026D500EF90E6517402F07BFF7A1079CF1229B39F
:1026E500D007D003D002D001D000D0D0D086D0847E
:0926F500D085D082D083D0E03200
:012FCD0032D1
:1026FE00C0E0C083C082C085C084C086758600C01D
:10270E00D075D000C000C001C002C003C0075391F5
:10271E00EF90E6557402F07BFF7A1079D31229B34D
:10272E00D007D003D002D001D000D0D0D086D08434
:09273E00D085D082D083D0E032B6
:012FCE0032D0
:10274700C0E0C083C082C085C084C086758600C0D3
:10275700D075D000C000C001C002C003C0075391AC
:10276700EF90E6517401F07BFF7A1079D71229B305
:10277700D007D003D002D001D000D0D0D086D084EB
:09278700D085D082D083D0E0326D
:012FCF0032CF
:10279000C0E0C083C082C085C084C086758600C08A
:1027A000D075D000C000C001C002C003C007539163
:1027B000EF90E6557401F07BFF7A1079DB1229B3B4
:1027C000D007D003D002D001D000D0D0D086D084A2
:0927D000D085D082D083D0E03224
:012FD00032CE
:012FD10032CD
:012FD20032CC
:1028AA00AB07AA06AC05E4FD903FD2E0600B7E00C0
:1028BA000DEE24EA12182BEAF0AE050D74EA2E1278
:1028CA00182BEBF0AF050D74EA2F12182BECF090D1
:1028DA003FC9E0FF7A3F7BEA122E0E903FC9E0FF24
:0328EA00022A2D92
:102A63008E408F418D428A438B44E4F545E545C34F
:102A7300954250200541E541AE407002054014FFE8
:102A8300E5442545F582E43543F583E0FD1228AAA4
:052A9300054580D92279
:102665008E428F438D448A458B46E4FDF547903F66
:10267500D2E06012E542FF7E000DEE24EAF582E429
:10268500343FF583EFF0AE050D74EA2EF582E434A0
:102695003FF583E543F0903FC9E0FF7A3F7BEA12BF
:1026A5002E0E903FC9E0FFAB46AA45AD44022DF280
:102DD500A210920790401F300707E4F01221F580FA
:0D2DE500067402F012215D122D35022E91B0
:0A2F5900A20F9210122DD5022E2AAD
:1026110090E67AE04401F0C2E990E678E04480F087
:1026210090E679741CF090E678E030E0F9EF441818
:1026310090E679F090E678E030E0F9EC90E679F018
:1026410090E678E030E0F9ED90E679F090E678E018
:102651004440F090E678E030E0F990E678E020E65A
:04266100F9D2E9229F
:092F6300054FE54F7002054E22F6
:021BCC00C10D49
:102C5C00903FCCEFF0F5CB8FCDAF05903FCDEFF0A3
:102C6C00F5CA8FCCE4F5C8758E19D2BDD2AFD2ADF2
:052C7C00D2CAF51F2281
:0D2F1800903FCCE0FF903FCDE0FD022C5C2F
:092F6C00A20E9211D20EA2112254
:092F7500A20E9212C20EA2122259
:032FAE00AF1F2230
:032FB100A20E224B
:102EEA00AD07AC06C3E49DFBE49CFFEBFD022C5C42
:052F9400C2CAC2AD221B
:03002B00022DB7EC
:102DB700C0E0300E0E300D04051F8007D20D122F14
:0E2DC70063C20D300203122F63C2CFD0E03280
:03004300021F0099
:03005300021F0089
:101F0000022CCA00022D9800022D7900022CEE004E
:101F1000022562000229F200022FB800022FB90048
:101F2000022FBA00022FBB00022FBC00022FBD00FF
:101F3000022C3700022FBE00021EB500022FBF0088
:101F4000021FB800022FB900022FC000022FC100EB
:101F5000022D5700022FC2000227D900022FC30012
:101F6000022FC400022FB900022FB900022FB900BE
:101F7000022FC500022FC600022FC700022FC80083
:101F8000022FC900022FCA00022FCB00022FCC0063
:101F90000226B500022FCD000226FE00022FCE0041
:101FA00002274700022FCF0002279000022FD00007
:081FB000022FD100022FD20024
:102B920090E682E030E004E020E60B90E682E0304E
:102BA200E119E030E71590E680E04401F07F147E01
:0C2BB2000012281F90E680E054FEF02284
:102C810090E682E044C0F090E681F04387010000C5
:042C9100000000221D
:102B6300300F0990E680E0440AF0800790E680E0A9
:102B73004408F07FDC7E0512281F90E65D74FFF0A9
:0F2B830090E65FF05391EF90E680E054F7F02278
:10281F008E358F3690E600E054187012E53624019D
:10282F00FFE43535C313F535EF13F536801590E614
:10283F0000E05418FFBF100BE53625E0F536E535FF
:10284F0033F535E5361536AE35700215354E600564
:06285F00122C9580EE2210
:082F8600E4F51BD2E9D2AF22F1
:102A2D0090E678E020E6F9C2E990E678E04480F09F
:102A3D00EF25E090E679F090E678E030E0F990E669
:102A4D0078E04440F090E678E020E6F990E678E012
:062A5D0030E1D6D2E922AF
:102B0000A90790E678E020E6F9E51B702390E678C7
:102B1000E04480F0E925E090E679F08D16AF03A956
:102B2000077517018A188919E4F51A751B01D32254
:022B3000C322BE
:102ACC00A90790E678E020E6F9E51B702590E678FA
:102ADC00E04480F0E925E0440190E679F08D16AFF2
:102AEC0003A9077517018A188919E4F51A751B03D0
:042AFC00D322C322FC
:03004B00021BCFC6
:101BCF00C0E0C083C082C085C084C086758600C057
:101BDF00D075D000C000C001C002C003C006C0074E
:101BEF0090E678E030E206751B06021CB990E678A5
:101BFF00E020E10CE51B64026006751B07021CB9AF
:101C0F00E51B24FE605F14603624FE7003021CAADD
:101C1F0024FC7003021CB624086003021CB9AB1726
:101C2F00AA18A919AF1A051A8F82758300121DEB16
:101C3F0090E679F0E51A65167070751B05806B904C
:101C4F00E679E0AB17AA18A919AE1A8E8275830030
:101C5F00121E18751B02E5166401704E90E678E0AF
:101C6F004420F08045E51624FEB51A0790E678E08B
:101C7F004420F0E51614B51A0A90E678E04440F0D7
:101C8F00751B0090E679E0AB17AA18A919AE1A8E4A
:101C9F0082758300121E18051A800F90E678E044B3
:101CAF0040F0751B008003751B005391DFD007D0E8
:101CBF0006D003D002D001D000D0D0D086D084D0AF
:081CCF0085D082D083D0E03201
:022BBE00A90765
:102BC000AE14AF158F828E83A3E064037017AD013E
:102BD00019ED7001228F828E83E07C002FFDEC3E88
:092BE000FEAF0580DF7E007F00DE
:012BE90022C9
:102DF200122ACCE51B24FA600E146006240770F335
:0C2E0200D322E4F51BD322E4F51BD322FD
:102E0E00122B00E51B24FA600E146006240770F3E3
:0C2E1E00D322E4F51BD322E4F51BD322E1
:102C95007400F58690FDA57C05A3E582458370F952
:012CA500220C
:102EFA0090E608E04401F043878075985AD29922F7
:102E7E001551A851A6073099FDC299A851E6F599AA
:032E8E00055122C9
:052F99007F0D022E7EF9
:102E6A00AE07EEC3940AEE5004243080022437FFE2
:042E7A00122E7E2274
:102ED900AD07EDC4540FFF122E6AED540FFF022EF9
:012EE9006A7E
:0E2F0A00AB07AA06AF02122ED9AF03022ED9D2
:1029B300155115511551A851A60308A60208A601E1
:1029C300A851860308E6FA08E6F9121DD26019A891
:1029D300518603080806E618860270010614F912E8
:0F29E3001DD2FF122E7E80D805510551055122BD
:0300000002231EBA
:0C231E00787FE4F6D8FD7581510223653C
:101DD200BB010689828A83E0225002E722BBFE020F
:091DE200E32289828A83E4932242
:101DEB00BB010CE58229F582E5833AF583E02250AD
:101DFB0006E92582F8E622BBFE06E92582F8E222F7
:0D1E0B00E58229F582E5833AF583E4932210
:101E1800F8BB010DE58229F582E5833AF583E8F000
:101E2800225006E92582C8F622BBFE05E92582C8AC
:021E3800F22294
:101E3A00BC000BBE0029EF8DF084FFADF022E4CC8C
:101E4A00F875F008EF2FFFEE33FEEC33FCEE9DEC55
:101E5A00984005FCEE9DFE0FD5F0E9E4CEFD22ED9B
:101E6A00F8F5F0EE8420D21CFEADF075F008EF2FE5
:101E7A00FFED33FD4007985006D5F0F222C398FDD6
:051E8A000FD5F0EA2273
:101E8F00D083D082F8E4937012740193700DA3A3E2
:101E9F0093F8740193F5828883E4737402936860F6
:061EAF00EFA3A3A380DFF6
:102E4100E4FFFE121DD2600C0FEF70010E09E97054
:052E5100F20A80EF22EF
:10232A0002228DE493A3F8E493A34003F68001F21A
:10233A0008DFF48029E493A3F85407240CC8C333B4
:10234A00C4540F4420C8834004F456800146F6DF83
:10235A00E4800B0102040810204080901A2EE47ECB
:10236A00019360BCA3FF543F30E509541FFEE49378
:10237A00A360010ECF54C025E060A840B8E493A33F
:10238A00FAE493A3F8E493A3C8C582C8CAC583CA6A
:10239A00F0A3C8C582C8CAC583CADFE9DEE780BE22
:011BCE000016
:00000001FF
